:1000000008308A0000280000FF00030E8301A100D1
:100010000A08A0008A010408A2007708A300780853
:10002000A4007908A5007A08A600831383128B1E0A
:100030001B280B1932288C308400001C21280C1836
:100040003528220884002308F7002408F800250832
:10005000F9002608FA0020088A00210E8300FF0E0E
:100060007F0E09008A110A1240288A110A124728B5
:100070000A108A100A11820728340C34013406341D
:10008000AD0A0319AE0A0B118A110A122128AB0A14
:100090000319AC0A2F122F08831687001030831221
:1000A0008706831608110430831288060C108A1103
:1000B0000A1221288C234D10E3377537F432721061
:1000C000D6182E18200520102019B01833104D26F0
:1000D00041210000C732E9336539AD267536EC326F
:1000E0007210C3377537F4327210D6182E18A00666
:1000F0000A00A83129103218B119A026CC204210CC
:1001000061376410D5295417633DA0060A000C001E
:10011000C3377537741D2536751020102010000068
:10012000491D2536751020102000A423CD2131173C
:100130003010253675102536751025367510A00639
:100140000A0046308400831300080319B4280230E3
:10015000F800F701F70BAA28F80BA9289730F70049
:10016000F70BB028800BA72808004D18B9280812F3
:10017000BA280816831608128312CD18C1288812CF
:10018000C22888168316881283124D19C9280813AD
:10019000CA280817831608138312CD19D12888138B
:1001A000D228881783168813000083120914831637
:1001B0000910DA28DB28831209108316091083122C
:1001C0000800CE018316081600308312081A013089
:1001D000CE048316881600308312881A0130F70087
:1001E0000310F70D7708CE0483160817003083122A
:1001F000081B0130F700F70DF70DFC30F705770805
:10020000CE048316881700308312881B0130F70054
:10021000F70DF70DF70DF830F7057708CE044E0807
:10022000F80008008316091089100911831289103B
:10023000831689100816881608178817831209155F
:100240008316091100008312091483160910000097
:100250008312E1207808CD000910831609100000F0
:10026000831209148316091035298312E1207808B6
:10027000CC0009108316091008128812081388137D
:1002800083124D0EF700F030F70577084C04F800A4
:100290007808CC00CC1F4E2983161A29CA08031DE2
:1002A0005329891054298914831689100000831258
:1002B0000911831609110000831209108316091011
:1002C00083124B0ECC000F30CC054C08CD00B5206E
:1002D0004B080F39CC00CD00B5200800831608125A
:1002E00088120813881309108910091183128910C4
:1002F00083168910831209118316091183120910BC
:10030000831609100F308312C600A1200130B900F6
:100310003908033C031C94290330CD00B520053077
:10032000C600A120B90A88290230CD00B520B90144
:100330003908033C031CA52939083820BA00CA0132
:100340003A08CB001221B90A98298A150A12B32853
:10035000470BAB29AE294030C800AF29C801013096
:100360004602C80748088038C900CA014908CB00BE
:10037000122108004508073A0319C8290B3A031946
:10038000CD29063A0319D529023A0319DB29E029B8
:100390000130C600C700A821E629CA010130CB0000
:1003A00012210230C600A120E6290130C600023029
:1003B000C700A821E629CA011030CB001221E62986
:1003C0000130CA004508CB001221E6290800831637
:1003D00003178C170C140000000083120C087F39DF
:1003E00003192B2A0313B90003170D080313BA00CE
:1003F00003170F080313BB003908C500BA213A08D8
:1004000003178D0003133B0803178F0083168C1707
:100410000C140000000083120C0D0E0D7F3903191F
:100420002B2A0313B90003170D080313BA0003178F
:100430000F080313BB003908C500BA213A08031797
:100440008D0003133B0803178F008D0A03198F0AD1
:100450000313E72903170313080083168613831277
:1004600086130830F800342A0000F817452AF813DC
:10047000C50C03188617031C86137817452A7813B2
:10048000F80B382A432A000086173F308400840B7B
:10049000472A0000F81B372A781B3F2A08008316DA
:1004A00003178C170C140000000083120C087F390E
:1004B0000319932A0313B90003170D080313BA0095
:1004C00003170F080313BB003908C5002D223A0893
:1004D00003178D0003133B0803178F0083168C1737
:1004E0000C140000000083120C0D0E0D7F3903194F
:1004F000932A0313B90003170D080313BA00031757
:100500000F080313BB003908C5002D223A08031752
:100510008D0003133B0803178F008D0A03198F0A00
:1005200003134F2A0317031308001030BF00F7010D
:10053000FA01BC0CBB0C031CA32A3D08F7070318E7
:10054000FA0A3E08FA07FA0CF70CF90CF80CBF0B84
:10055000992A8A150A1202298E30F7004008F800FD
:100560003F08F900FA01F808031DC02A7908F800CD
:10057000F9010830F702F808031DC02AF701C82A5C
:100580000310F81BC72AF90DF80DF703C02AF8135A
:1005900008003B080319392BC3003F080319392B06
:1005A000C3070318DA2A7F30C302031C392B03194F
:1005B000392BDE2A8130C3070318392B4308F70093
:1005C000F801F901FA013C08C700C7173D08C60049
:1005D0003E08C5001830C300C401451C072B420863
:1005E000FA07031CF92AF90A031DF92AF80A031964
:1005F000C4174108F907031C002BF80A0319C41794
:100600004008BD00BD173D08F8070318C417C40D06
:10061000F80CF90CFA0CC70CC60CC50C0310C30B74
:10062000EC2A0130F7070318392BF81B1E2BC70DD6
:10063000FA0DF90DF80DF7030319392BC71F2F2BEE
:10064000FA0A031D2F2BF90A031D2F2BF80A031D8D
:100650002F2BF80CF90CFA0CF70A0319392B3C086C
:10066000C4004008C406C41F372BF8173D2BF813ED
:100670003D2BF701F801F901FA018A150A12302918
:1006800080308318C406C901CA014008C800440864
:10069000C8063F080319302CC700F70043080319A8
:1006A000392CC7020319D52B031C932B4408CD000A
:1006B000CD174508CC004608CB00CA010310CD0C6D
:1006C000CC0CCB0CCA0CC70B5D2BC81F6A2B491472
:1006D0004D2C491047104916423084008313622C78
:1006E0004912C81B7D2B471C882BCD0CCC0CCB0C86
:1006F000CA0CF70A0319482C882BCD1B8B2B03102F
:10070000CA0DCB0DCC0DCD0DF7030319482C7D2B55
:100710004917F52B49134008C800C81F912BCD1766
:10072000412CCD13412C4308C700F7003F08C702F6
:100730004008CD00CD174108CC004208CB00CA01CB
:100740000310CD0CCC0CCB0CCA0CC70B9F2BC81FB5
:10075000AC2BC9144D2CC9104710C9164630840063
:100760008313622CC912C81BBF2B471CCA2BCD0C8C
:10077000CC0CCB0CCA0CF70A0319482CCA2BCD1B86
:10078000CD2B0310CA0DCB0DCC0DCD0DF7030319E6
:10079000482CBF2BC917F52BC9134408C800C81F24
:1007A000D32BCD17412CCD13412C4408CD00CD17B0
:1007B0004508CC004608CB00C81FE22BCD134915D5
:1007C0004D2C4911CA014710423084008313622C1A
:1007D000C81B0B2C4008C800471CF52BCD0CCC0CBB
:1007E000CB0CCA0CF70A0319482CCA1F062CCB0ADB
:1007F000031D062CCC0A031D062CCD0A031D062C56
:10080000CD0CCC0CCB0CF70A0319482C491B8A2BB6
:10081000C91BCC2B2A2C8030CD06CD1F132C4D2C80
:100820004408C800202C4008C800CD08031D202C17
:10083000CC08031D202CCB08031D202CF701412CD4
:10084000CD1B2A2C0310CA0DCB0DCC0DCD0DF70BF3
:10085000202C482CC81F2E2CCD17412CCD13412CF9
:100860004308F7004408CD004508CC004608CB00FB
:10087000412C3F08F7004008CD004108CC00420859
:10088000CB004D08F8004C08F9004B08FA00802C0A
:10089000F701F801F901FA01802CCA01CB09CC0952
:1008A000CD09CA09CA0A031D5B2CCB0A031D5B2CA8
:1008B000CC0A0319CD0A4918692BC918AB2B491961
:1008C000E12B102C0008CB07031C6C2CCC0A031D59
:1008D0006C2CCD0A0319471484030008CC07031CB1
:1008E000742CCD0A0319471484030008801F803A32
:1008F000CD0703184714491A702BC91AB22BE82BDD
:100900008A150A1253298E30F7003F08F702400873
:10091000F9004108F800F917F70803199A2C031099
:10092000F908031D962CF80803199A2CF90CF80CF9
:10093000F70B8F2CC01FA12CF809F909F80A03192D
:10094000F90A8A150A125E29831603178C170C14EC
:10095000000000000318D32C83120C087F39031306
:10096000BA0003170D080313BB0003170F08031386
:10097000BC003A08C500BA213B0803178D000313D9
:100980003C0803178F0083168C170C14000000001E
:1009900083120313B90BCD2CD02C83160317D32C41
:1009A000F22C8316031783120C0D0E0D7F390313DF
:1009B000BA0003170D080313BB0003170F08031336
:1009C000BC003A08C500BA213B0803178D00031389
:1009D0003C0803178F008D0A03198F0A03100313B5
:1009E000B90BA42C0800F701F801F901FA01CD01B7
:1009F000CE01CF01D0014C084B044A04490403192D
:100A0000312D2030D1000310C50DC60DC70DC80D06
:100A1000CD0DCE0DCF0DD00D4C085002031D1A2D5B
:100A20004B084F02031D1A2D4A084E02031D1A2DB2
:100A300049084D02031C2B2D4908CD024A08031C0E
:100A40004A0FCE024B08031C4B0FCF024C08031C6D
:100A50004C0FD0020314F70DF80DF90DFA0DD10B60
:100A6000032D4D308400831308000408BD003B3083
:100A7000C4009A30C300CA30C200C1010A30BF00AE
:100A80003C08C8003B08C7003A08C6003908C50042
:100A90004408CC004308CB004208CA004108C90002
:100AA000F3240008B900840A0008BA00840A000888
:100AB000BB00840A0008BC00F708031D722D3F0824
:100AC000013A0319722D3D080319732D0F393F02A6
:100AD00003196C2D0318782DBD1B782D3D1B732D2C
:100AE0002030742DBD013030F7077708C500BA21DA
:100AF0004408C8004308C7004208C6004108C500B2
:100B0000CC01CB01CA010A30C900F3247A08C40021
:100B10007908C3007808C2007708C100BF0B402DD8
:100B20008A150A12A629C1010408C0004110831BBE
:100B300041143A0EF038BC00BC07E23EBD00323E24
:100B4000BF003A080F39BD07BD07BF07E93EBE0029
:100B5000BE07BE07390E0F39BE07BF07BE0DBF0D5A
:100B6000BF09BF0D39080F39BF07BC0D0730BB00E7
:100B70000A30BF07BE03031CB92DBE07BD03031C0B
:100B8000BD2DBD07BC03031CC12DBC07BB03031C4B
:100B9000C52D3B3084008313073040054013840784
:100BA0003F300402031940170008F700031DE02D31
:100BB000401BE02D401AF22DC019E02D2030E32D0E
:100BC000C01540123030F707BA010408B9003A10D6
:100BD000831B3A147708C500BA21390884008313AF
:100BE0003A188317840A401FD02D08000830C0022D
:100BF000031C062E4030840083130310800C000871
:100C00000319062E042E0000800B032E0800BC01E1
:100C10003C083902031C4F2E83160811043083123E
:100C20008806BE010130BD003B08C0003A08BF0085
:100C3000F801F901F701FA014008031D222E3F08CF
:100C400003193C2E1030C1000310BD0DBE0DF70D71
:100C5000FA0D40087A02031D2F2E3F087702031C6D
:100C6000382E3F08F702031CFA034008FA02031467
:100C7000F80DF90DC10B242E7908BE007808BD00CF
:100C80003E08BF00BF0ABF0303194A2EFF30C00051
:100C9000F625432E3D08C000F625BC0A082E0800A4
:100CA000831603178C170C140000000003187F2E06
:100CB00083120C087F390313BA0003170D080313BE
:100CC000BB0003170F080313BC003A08C5002D2210
:100CD0003B0803178D0003133C0803178F0083168E
:100CE0008C170C140000000083120313B90B792E2B
:100CF0007C2E831603177F2E9E2E831603178312D6
:100D00000C0D0E0D7F390313BA0003170D080313E2
:100D1000BB0003170F080313BC003A08C5002D22BF
:100D20003B0803178D0003133C0803178F008D0A3F
:100D300003198F0A03100313B90B502E0800C101C9
:100D40000408C0004110831B41143A0EF038BC0067
:100D5000BC07E23EBD00323EBF003A080F39BD0776
:100D6000BD07BF07E93EBE00BE07BE07390E0F39FB
:100D7000BE07BF07BE0DBF0DBF09BF0D39080F3934
:100D8000BF07BC0D0730BB000A30BF07BE03031C02
:100D9000C52EBE07BD03031CC92EBD07BC03031C23
:100DA000CD2EBC07BB03031CD12E3B308400831324
:100DB00007304005401384073F30040203194017F1
:100DC0000008F700031DEC2E401BEC2E401AFE2EEF
:100DD000C019EC2E2030EF2EC01540123030F7072E
:100DE000BA010408B9003A10831B3A147708C50009
:100DF0002D223908840083133A188317840A401F70
:100E0000DC2E08000408BD003B30C4009A30C3004B
:100E1000CA30C200C1010A30BF003C08C8003B080C
:100E2000C7003A08C6003908C5004408CC0043088A
:100E3000CB004208CA004108C900F3240008B900E9
:100E4000840A0008BA00840A0008BB00840A00086B
:100E5000BC00F708031D3F2F3F08013A03193F2F3D
:100E60003D080319402F0F393F020319392F03188A
:100E7000452FBD1B452F3D1B402F2030412FBD016D
:100E80003030F7077708C5002D224408C800430812
:100E9000C7004208C6004108C500CC01CB01CA0109
:100EA0000A30C900F3247A08C4007908C30078081E
:100EB000C2007708C100BF0B0D2F8A150A12482AFD
:10100000840183131F308305713083168F000F080E
:10101000861383128617AA01A901A801A701AC01B2
:10102000AB01AE01AD01831603170908C039890071
:1010300003131F129F1200300317880083128701C9
:1010400088018901FF300313AF00B1013C30B000CB
:10105000B801B701831603170908C03989000313C3
:101060001F129F12013003178800831203131F13EE
:101070009F1783169F1783121F149412AF122F0805
:101080008316870083122F162F088316870083127A
:10109000AF112F08831687000130831294000030AF
:1010A000831694000108C039073881000730831285
:1010B00090000030F80092000030831692008312F6
:1010C0002F112F0883168700831207118316091327
:1010D0000C308312970083169B019C0101309D0008
:1010E0008312AF102F0883168700831287100C30ED
:1010F0009D0001308000713083168F000F0883122D
:1011000095019B012F132F08831687008312071761
:10111000AF122F0883168700831287162F122F080D
:101120008316870083120716831688118312881589
:10113000831608118312081103178701A430880051
:10114000103089008316031385120514863097002A
:101150008D1683128B1683160C148C14C0308312D8
:101160008B048A116E298A155A3003178D000030BE
:101170008F008A110313E7218A156A3003178D0047
:1011800000308F008A1103134F228A15793003171C
:101190008D0000308F008A1103134F228A1504300E
:1011A000B900FA30C6008A11A1208A15B90BD128DE
:1011B000873003178D0000308F008A110313E72159
:1011C0008A150D30C5008A112D228A150A30C500F6
:1011D0008A112D228A158F018E010F08FA000E0840
:1011E000F7000F087A02031DED287708B9007A0886
:1011F000BA00FF30BC00BB002C08BE002B08BD00AD
:101200008A11952A8A157908FA0078083907A70003
:101210003A08A8007A0803187A0FA807A901AA01BA
:1012200001303007B9003108BA000318BA0A2E0895
:10123000C0002D08BF008A11AC228A157A08BE00B2
:101240007908BD007808BC007708BB006F30C20089
:10125000F030C1000530C0007A30BF008A11C92AC1
:101260008A157708BB007808BC007908BD007A08A9
:10127000BE003A08C0003908BF008A11AC228A15A6
:1012800083147A08C2007908C1007808C000770882
:10129000BF003E08C6003D08C5003C08C4003B082E
:1012A000C3008A11402B8A157A08C2007908C10050
:1012B0007808C0007708BF008A11832C8A15790846
:1012C000B3007808B2000F08FA000E08F7000F0804
:1012D0007A02031D63297708B9007A08BA00340836
:1012E0003902031D772935083A0203198829831624
:1012F00008110430831288060F08FA000E08F70060
:101300000F087A02031D7C297708B4007A08B5001B
:101310000130C600C7008A11A8218A15883003173A
:101320008D0000308F00031006300313B9008A11BE
:10133000A4248A15413084002A08BC002908BB0077
:101340002808BA002708B9008A11352D8A158C3073
:1013500003178D0000308F00031405300313B9000C
:101360008A11A4248A150130C6000230C7008A11F0
:10137000A8218A155430C5008A11BA218A153A303D
:10138000C5008A11BA218A15103084003308BA00CA
:101390003208B9008A1193258A152030C5008A11B8
:1013A000BA218A152030C5008A11BA218A15203049
:1013B000C5008A11BA218A150930C6000230C7005B
:1013C0008A11A8218A154930C5008A11BA218A15C7
:1013D0003A30C5008A11BA218A15103084003108CC
:1013E000BA003008B9008A1193258A159230031784
:1013F0008D0000308F00031404300313B9008A11EC
:10140000A4248A15B208031D5C2AB308031D5C2AB4
:101410008101AE01AD01E830B9000230BB00BC3043
:10142000BA008A1107268A15953003178D000030FF
:101430008F00031008300313B9008A1150268A1553
:10144000103084003808BA003708B9008A119F2686
:101450008A152030C5008A112D228A15103084008B
:101460003108BA003008B9008A119F268A15203049
:10147000C5008A112D228A15413084002A08BC003B
:101480002908BB002808BA002708B9008A11022FD2
:101490008A159E3003178D0000308F00031404302E
:1014A0000313B9008A1150268A158F018E01AC01F1
:1014B000AB01B70A0319B80A3618072B2F152F08E6
:1014C0008316870083120719892A1430C6008A11EF
:1014D000A1208A152F152F0883168700831207195C
:1014E000892A36146430B9000230BB00BC30BA001F
:1014F0008A1107268A153108FF3C031C892A031D1F
:10150000852A3008F93C031C892A0530B0070318E6
:10151000B10AAF152F088316870083128719BD2AD9
:101520001430C6008A11A1208A15AF152F08831622
:10153000870083128719BD2A36146430B90002303F
:10154000BB005830BA008A1107268A153108FF3CC3
:10155000031CB62A031DB02A3008F93C031CB62A26
:101560000530B0020030031C0130B1028101AE0130
:10157000AD018F018E01AC01AB01831608148312FB
:101580000818DE2A1430C6008A11A1208A15831695
:10159000081483120818DE2A36146430B9000130AA
:1015A000BB00F430BA008A1107268A15300FDB2AF7
:1015B000310FDB2ADE2AB00A0319B10A8316881418
:1015C00083128818072B1430C6008A11A1208A15AF
:1015D0008316881483128818072B36146430B900D8
:1015E0000130BB009030BA008A1107268A15300FEF
:1015F000FC2A310FFC2A002B30080319B103B00379
:101600008101AE01AD018F018E01AC01AB012F153F
:101610002F08831687008312071D202BAF152F0874
:10162000831687008312871D202B831608148312CC
:10163000081C202B831688148312881C202B36103C
:04164000ED2863002E
:04400E00F52CFF3F4F
:00000001FF
